:100000000AC023C022C021C020C01FC01EC01DC006
:100010001CC01BC01AC011241FBECFEDCDBF10E005
:10002000A0E6B0E0EEE0F1E003C0C89531960D9295
:10003000A036B107D1F710E0A0E6B0E001C01D92F4
:10004000A036B107E1F710D061C0DACFCF93DF93CC
:10005000CDB7DEB7E2E3F0E01082E1E3F0E08AE062
:100060008083DF91CF910895CF93DF93CDB7DEB733
:1000700024970FB6F894DEBF0FBECDBFA2E3B0E069
:10008000E2E3F0E0808188608C938AE090E09C83DA
:100090008B8313C080E395E79A83898305C08981A8
:1000A0009A8101979A83898389819A810097B9F708
:1000B0008B819C8101979C838B838B819C81009792
:1000C00049F7A2E3B0E0E2E3F0E0908187EF892313
:1000D0008C938AE090E09C838B8313C080E395E748
:1000E0009A83898305C089819A8101979A8389833C
:1000F00089819A810097B9F78B819C8101979C83B4
:0E0100008B838B819C81009749F7B8CFFFCF8E
:00000001FF
